:100000008A110A120528000009000730990083169A
:100010000510851005118312BC30A0000230A1002C
:1000200086212F20AC012C081E3C031C2B28AD017F
:100030002D083B3C031C2528E830A0000330A1001C
:1000400086210130AD07031C18281F3083050130BD
:10005000AC07031C13281F3083050C282E28051419
:100060005830A0000230A1008621BA202E21AC20F9
:100070002E21E2202E2160202E21A2202E2185205B
:100080002E2115212E219E202E212E21AC202E2125
:1000900058202E219E202E2170202E2158202E21E6
:1000A000A2209030A0000130A10086210510080098
:1000B000522163210800632152215221522108005C
:1000C00063215221632152210800632152215221D0
:1000D00008005221080052215221632152210800B8
:1000E00063216321522108005221522152215221C1
:1000F000080052215221080052216321632163210B
:1001000008006321522163210800522163215221FA
:100110005221080063216321080063215221080055
:10012000632163216321080052216321632152214D
:1001300008006321632152216321080052216321B9
:100140005221080052215221522108006321080047
:100150005221522163210800522152215221632150
:10016000080052216321632108006321522152219A
:100170006321080063215221632163210800632168
:1001800063215221522108006321632163216321ED
:100190006321080052216321632163216321080048
:1001A00052215221632163216321080052215221EF
:1001B00052216321632108005221522152215221F0
:1001C000632108005221522152215221522108005C
:1001D00063215221522152215221080063216321BF
:1001E00052215221522108006321632163215221AF
:1001F00052210800632163216321632152210800F9
:10020000522163215221632152216321080063217D
:10021000632152215221632163210800522152217E
:10022000632163215221522108006321522152216E
:10023000632152210800632152215221522163215E
:1002400008006321522152215221522163210800CA
:1002500005116430A000A101862108000511643059
:10026000A000A10186216430A000A1018621643094
:10027000A000A1018621080005116430A000A101A1
:1002800086216430A000A10186216430A000A10174
:1002900086216430A000A10186216430A000A10164
:1002A000862108000515053084000230AA00993027
:1002B000A0000230A1004430A2000030A300C12100
:1002C0000511282108000515053084000230AA0018
:1002D0009930A0000230A1000E30A2000130A3002E
:1002E000C1210511282108000515053084000230C0
:1002F000AA009930A0000230A100EE30A200023026
:10030000A300C1210511282108008529A00803198F
:1003100091299821A00300000000000000000000C7
:100320008629A108031908009821A103A0038629A2
:100330000C30A500A50B9A29000000001230A20085
:10034000A20BA729A921A921000000000800A921CA
:10035000A0290D30A400A40BAB2900000800103028
:10036000A8020001031C013EA902031C0800B829D1
:100370000A30A8020001031C013EA902031C080068
:10038000B8292A0880042008A8002108A900AF2164
:100390000130A202031CA3032A0980052008A8003B
:1003A0002108A900AF21A208031DC129A308031D2C
:0403B000C129080057
:02400E00C431BB
:00000001FF
